:020000040800F2
:1000000000040020E1010008ED0D0008F10D0008DA
:10001000450E0008F10D0008190E0008E301000864
:10002000E3010008E3010008E3010008E92E0008ED
:10003000E3010008E3010008E3010008E301000810
:10004000E3010008E3010008E3010008E301000800
:10005000E3010008E3010008493100087531000898
:10006000A1310008CD310008F9310008E301000892
:10007000E3010008E3010008E3010008E3010008D0
:10008000E3010008E3010008E3010008E3010008C0
:10009000E3010008E3010008E3010008253200083D
:1000A000E3010008E3010008E3010008E3010008A0
:1000B000652F0008E3010008E3010008E3010008E0
:1000C000E3010008E3010008E3010008E301000880
:1000D000E3010008E3010008E3010008E301000870
:1000E0008D320008E3010008E3010008E301000885
:1000F000E3010008E3010008E3010008E301000850
:10010000E3010008E3010008E3010008E30100083F
:10011000E3010008E3010008E3010008E30100082F
:10012000E3010008E3010008E3010008E30100081F
:10013000E3010008E3010008E3010008E30100080F
:10014000E3010008E3010008E3010008412600087C
:10015000E3010008E3010008E3010008E3010008EF
:10016000E3010008E3010008E3010008E3010008DF
:10017000E3010008E3010008E3010008E3010008CF
:10018000E3010008E3010008E3010008E3010008BF
:10019000E3010008E3010008E3010008E3010008AF
:1001A000E3010008E3010008E3010008E30100089F
:1001B000E3010008E3010008E3010008E30100088F
:1001C000E3010008E3010008E3010008E30100087F
:1001D000E3010008E3010008E3010008E30100086F
:1001E00002E000F000F8FEE772B6394880F30888B4
:1001F000384880F3098838484EF60851CEF200019D
:10020000086040F20000CCF200004EF63471CEF2ED
:1002100000010860BFF34F8FBFF36F8F40F2000003
:10022000C0F2F0004EF68851CEF200010860BFF334
:100230004F8FBFF36F8F4FF00000E1EE100A4EF6C4
:100240003C71CEF200010860062080F31488BFF3F1
:100250006F8F01F0BDFE02F0DDFD4FF055301F49FC
:100260001B4A91423CBF41F8040BFAE71C49194A6A
:1002700091423CBF41F8040BFAE71A491A4A1B4B5A
:100280009A423EBF51F8040B42F8040BF8E70020F5
:100290001749184A91423CBF41F8040BFAE701F0B4
:1002A0009BFE02F013FE144C144DAC4203DA54F8DA
:1002B000041B8847F9E700F03FF8114C114DAC42A0
:1002C00003DA54F8041B8847F9E701F083BE000005
:1002D000000400200024002000000008000000208E
:1002E00000040020A036000800240020282400205C
:1002F0002824002018300020E0010008E001000858
:10030000E0010008E00100082DE9F04F2DED108A12
:10031000C1F80CD0C3689D46BDEC108ABDE8F08FD3
:10032000002383F311882846A047002001F0DAFA61
:1003300001F09EFA00DFFEE71A4B6FF0700270B515
:1003400000241A700F225C709C70DC701C715C7150
:100350009C71DC711C725C729A72DC7201F00AFE94
:10036000064601F02FFE054650B90F4B9E4217D0AE
:1003700001339E4241F2883412BF05460024012514
:10038000002001F001FE0DB100F0B2F800F002FD16
:1003900000F0E8FB204600F005F900F0A9F8F9E7C5
:1003A0000446EDE728240020010007B008B500F05E
:1003B0007BFBA0F120035842584108BD07B5054B0F
:1003C00002211B88ADF8043001A800F0BBFB03B08C
:1003D0005DF804FB70330008064991F8243033B10E
:1003E00000230822086A81F8243000F0DDBB0120D8
:1003F000704700BF482400202DE9F84F224C1646D4
:1004000094F824200746884682BBDFF87C90002EB3
:1004100038D094F824A0BAF1000F05D12022FF2192
:100420004846276200F0A4FCCAF10805B54228BF7F
:1004300035465FFA85FBAD0041462A4604EB8A004B
:1004400000F06EFC94F82430A6EB0B069B445FFA98
:100450008BFBBBF1080F2F44A844F6B284F824B0FC
:10046000D5D1FFF7B9FF0028D1D108E0236A03EB0B
:1004700082038342C9D0FFF7AFFF0028C5D1002017
:10048000BDE8F88F0120FBE74824002010B52023A9
:1004900083F311881248C3680BB101F0A9FA002355
:1004A000104A0F484FF47A7101F066FA002383F383
:1004B00011880D4C236813B12368013B23606368E6
:1004C00013B16368013B6360084B1B7833B9636801
:1004D00023B9022000F01AFC3223636010BD00BF74
:1004E000342400208D04000878250020702400208A
:1004F00010B5244B244A1968013142D00433934289
:10050000F9D1224C224B22689A423AD9214B9B685E
:1005100003F1006303F580339A4232D2002000F0E9
:100520003BFB1D4B0220187000F0E8FB1B4B1A6CC4
:1005300000221A64196E1A66196E596C5A64596E43
:100540005A665A6E5A6942F080025A615A6922F01C
:1005500080025A615A691A6942F000521A611A6996
:1005600022F000521A611B6972B60D4A054B1360E6
:100570001B682268202181F311889D4683F3088837
:10058000104710BD00000108200001080400010808
:10059000FFFF0008282400207024002000380240BB
:1005A00008ED00E02DE9F04F99B0B14C0190202208
:1005B000FF2110A8A66800F0DBFBAE4A1378A34623
:1005C000A3B9AD480121C3601170202383F31188C2
:1005D000C3680BB101F00CFA0023A84AA6484FF4F7
:1005E0007A7101F0C9F9002383F31188019B13B1DB
:1005F000A34B019A1A60A34AA149019F02920023CA
:1006000013704B6099461D461C469846012000F029
:1006100075FB27B19A4B1B68002B00F00F8200205E
:1006200000F042FA0490049B002BF2DB012000F062
:100630005BFB049B213B122BE8D801A252F823F06C
:100640008D060008B5060008250700080D060008FD
:100650000D0600080D060008B9070008A9090008E2
:100660009D080008090900083B09000869090008FD
:100670000D060008810900080D060008FB090008A6
:10068000A70700080D060008430A00080220FFF72C
:100690008DFE002840F0FD81019BB9F1000F08BFDD
:1006A0001F46794B1B88ADF82C3002210BA800F0B7
:1006B00049FAABE74FF47A7000F0F6F9031E0393A2
:1006C000EADB0220FFF772FE82460028E4D0039B9B
:1006D000581E042800F2DF81DFE800F0030E111439
:1006E000170018A8052340F8343D042100F02AFA29
:1006F00055464FF0000856E004215D48F6E7042116
:100700006248F3E704216248F0E71C25284600F020
:1007100045FA04350B9004210BA800F013FA2C2D98
:10072000F4D1E5E7002CB7D0002DB5D00220FFF7BB
:100730003DFE0446002800F0B1810120514D00F03B
:100740002BFA0220287000F0D9FA4FF000095FFA66
:1007500089FA504600F030FA074658B1504600F08A
:100760003BFA09F101090028F1D12546A1460027ED
:10077000484B97E7012302202B7000F0B5FA3E4664
:10078000DBF80830B34206D9304600F007FA0130F2
:10079000EBD10436F4E7029B00261E70384BA146CD
:1007A0005E602546374600F0EBFA14B1002D18BF05
:1007B0000027FFF703FE29E7002C3FF46DAF002D63
:1007C0003FF46AAF029B0220187000F097FA3220C3
:1007D00000F06AF9B0F1000AC0F260811AF0030477
:1007E00040F05C81DBF808200AEB0603934200F23C
:1007F0005581BAF5807F00F25181A2450DDD4FF49D
:100800007A7000F051F90490049B002BC0F24681ED
:10081000214A049BA3540134EFE7C820FFF7C6FD2B
:100820000446002800F03A811F2E11D8C6F1200599
:10083000554528BF554610AB26F003002A461649F9
:10084000184400F06DFA2A46FF21134800F090FA90
:100850004FEAAA0A5FFA8AF20F493046FFF7CCFD49
:100860000546002800F01C8106EB8A0604469AE73C
:100870002824002074250020342400208D04000842
:100880007825002070240020723300082C240020DA
:100890003024002074330008742400200220FFF765
:1008A00085FD00283FF4F8AEFFF796FD00283FF4E1
:1008B000F3AE4FF0000A5346DBF8082052451CD92E
:1008C000BAF11F0F12D8109A01320FD02AF003028A
:1008D00018A90A4452F8202C0B92184604220BA99E
:1008E00000F0C4FA0AF1040A0346E5E75046039310
:1008F00000F054F9039B0B90EFE718A8042140F88F
:100900004C3D00F01FF94EE718A8002340F8343D95
:10091000642100F0F3F800287FF4BEAE0220FFF758
:1009200045FD00283FF4B8AE0B9800F067F918AB0E
:1009300043F8480D04211846E3E718A8002340F8BF
:10094000343D642100F0DAF800287FF4A5AE0220DF
:10095000FFF72CFD00283FF49FAE0B9800F05CF9E8
:1009600018AB43F8440DE5E70220FFF71FFD002810
:100970003FF492AE00F056F918AB43F8400DD9E7BA
:100980000220FFF713FD00283FF486AE0BA91420C8
:1009900000F04EF9824618A8042140F83CAD00F062
:1009A000D1F851460BA8ACE7322000F07DF8B0F149
:1009B000000AFFF671AE1AF0030F7FF46DAEDBF89C
:1009C00008200AEB080393423FF666AE0220FFF7C9
:1009D000EDFC00283FF460AE2AF0030AC244C24591
:1009E0003FF4E1AE404600F0D9F804210A900AA88D
:1009F00000F0A8F808F10408F1E74FF47A70FFF767
:100A0000D5FC00283FF448AEFFF7E6FC00283FF491
:100A1000AFAE109B01330CD0082210A90020FFF7C5
:100A2000EBFC00283FF4A4AE2022FF2110A800F028
:100A30009FF9FFF7C3FC1B4800F05AFF19B0BDE84F
:100A4000F08F002C3FF428AE002D3FF425AE18A8FF
:100A5000002340F8343D642100F050F8824600281D
:100A60007FF41AAE0220FFF7A1FC00283FF414AE79
:100A70000390FFF7A3FC41F2883000F039FF0B9898
:100A800000F0B2F900F07CF9039B57461D461C4666
:100A9000BCE5044687E64FF00008FDE52C46FBE583
:100AA000254665E6A086010037B5114B1A7801325C
:100AB000D2B20024012A01468DF8074011D80D4812
:100AC00003681D6A4FF47A734B4301220DF107014D
:100AD000A847012805D1084B9DF807001C7003B0FA
:100AE00030BD4FF4FA7000F003FF4FF0FF30F6E72F
:100AF00000240020482600208425002038B50E4B15
:100B00001A780132D2B2012A05460ED80B48036882
:100B10001C6A4FF47A734B4304222946A0470428E9
:100B200003D1074B0020187038BD4FF4FA7000F065
:100B3000DFFE4FF0FF30F7E70024002048260020BA
:100B40008425002030B4054C2368DD69044B0A4637
:100B5000AC460146204630BC604700BF4826002016
:100B6000A086010070B501F009F9094C094E20700A
:100B7000002530682378834208D901F0F9F83368FA
:100B800005440133B5F5803F3360F2D370BD00BF3B
:100B9000852500208025002001F09EB900F100602D
:100BA00000F580300068704700F10060920000F5A9
:100BB000803001F029B90000054B1A68054B1B78FD
:100BC0009B1A834202D9104401F0D2B8002070472A
:100BD000802500208525002038B5074D044628686B
:100BE000204401F0CDF828B928682044BDE83840F9
:100BF00001F0DEB838BD00BF8025002010F00303EF
:100C000008D1B0F5007F05D800F10050A0F50840EC
:100C10000068704700207047014BC058704700BF04
:100C2000107AFF1F014B1868704700BF002004E0D6
:100C3000F0B52A4B1A68C2F30B03120C63B140F2F1
:100C40001344A34231D040F21944A3422FD040F2C2
:100C50002144A3422DD10323214C0C2505FB034342
:100C60005E6893F9083042F20104A24224D0B2F542
:100C7000805F23D041F20104A24221D041F203045B
:100C8000A2421FD041F20704A24208BF3123451EF1
:100C90000D44013E0A46AA421ED216F9017F541C99
:100CA00097B104F8017C2246F5E70123D4E702233B
:100CB000D2E73F230B4ED6E73323E3E74123E1E7B7
:100CC0005A23E4E75923E2E72C20A542107001D90A
:100CD000941C5370601AF0BD1446FBE7002004E03A
:100CE0008433000878330008022802BF024B4FF417
:100CF00000129A61704700BF00040240022802BF40
:100D0000014B20229A61704700040240022801BF73
:100D1000024A536983F02003536170470004024084
:100D200010B50023934203D0CC5CC4540133F9E7DF
:100D300010BD000030B5441E14F9010F0B4640B140
:100D400093F90050854201F1010102D112B1013A3B
:100D5000F2E71AB193F90020801A30BD1046FCE783
:100D600002460346981A13F9011B0029FAD170476D
:100D700002440346934202D003F8011BFAE770478E
:100D8000024B1A78024B1A70704700BF842500206E
:100D90000024002038B5104D104C284600F004F90E
:100DA0002146284600F02CF924680D48626DD2F8DF
:100DB000043843F00203C2F8043800F099FD0949F1
:100DC000204600F021FA626DD2F8043823F00203C5
:100DD000C2F8043838BD00BF48260020503400084F
:100DE00040420F007834000870470000FEE7000022
:100DF00000B59BB0EFF3098168226846FFF790FFCA
:100E0000EFF30583034B9A6B9A6A9A6A9A6A9A6A15
:100E10009B6AFEE700ED00E000B59BB0EFF30981AF
:100E200068226846FFF77CFFEFF30583044B9A6B5B
:100E30009A6A9A6A9A6A9A6A9A6A9B6AFEE700BFF5
:100E400000ED00E000B59BB0EFF309816822684631
:100E5000FFF766FFEFF30583034B5A6B9A6A9A6AB2
:100E60009A6A9A6A9B6AFEE700ED00E030B5094D88
:100E70000A4491420DD011F8013B5840082340F339
:100E80000004013B2C4013F0FF0384EA5000F6D12C
:100E9000EFE730BD2083B8ED002304491A465A50CD
:100EA000C8180833802B4260F9D17047882500208C
:100EB000026843681143016003B11847704700009E
:100EC00013B5446BD4F894341A681178042915D1F9
:100ED000217C022912D11979128901238B401342F6
:100EE0000CD101A904F14C0001F010FED4F8944497
:100EF000019B21790246206800F0D2F902B010BDB2
:100F0000143001F093BD00004FF0FF33143001F0B6
:100F10008DBD00004C3001F065BE00004FF0FF3386
:100F20004C3001F05FBE0000143001F061BD0000E4
:100F30004FF0FF31143001F05BBD00004C3001F088
:100F400031BE00004FF0FF324C3001F02BBE0000EC
:100F5000D0F8942438B5136819780429054601D0CF
:100F6000012038BD017C0229FAD112795C89012067
:100F700090400440F4D105F1140001F0F3FC024666
:100F80000028EDD0D5F894544FF48073286869791F
:100F900000F074F92046E4E7406BFFF7D9BF00008A
:100FA00000207047704700007FB5124B036000239C
:100FB0004360C0E90233012502260F4B0574044645
:100FC0000290019300F18402294600964FF4807349
:100FD000143001F0A3FC094B0294CDE9006304F541
:100FE00023724FF48073294604F14C0001F06AFD2E
:100FF00004B070BDD4330008990F0008C10E00087A
:101000000B68202282F311880A7903EB8202906137
:101010004A79093243F822008A7912B103EB82033C
:10102000986102230374C0F89414002383F3118899
:101030007047000038B5037F044613B190F8543070
:10104000ABB9201D01250221FFF732FF04F1140086
:1010500025776FF0010100F073FC84F8545004F11F
:101060004C006FF00101BDE8384000F069BC38BDAC
:1010700010B5012104460430FFF71AFF002323773F
:1010800084F8543010BD000038B5044600251430F3
:1010900001F05CFC04F14C00257701F02BFD201DD4
:1010A00084F854500121FFF703FF2046BDE8384083
:1010B000FFF74EBF90F8443003F06003202B07D1B8
:1010C00090F84530202B03D3212B03D9222B09D0B4
:1010D00000207047054B83630723C3630023036429
:1010E000012070470023C0E90E33F8E701240020F7
:1010F000D0F8943437B51A681178042904461AD107
:10110000017C022917D11979128901238B401342DE
:1011100011D100F14C05284601F0ACFD58B101A9F0
:10112000284601F0F3FCD4F89444019B217902464F
:10113000206800F0B5F803B030BD000000EB81037B
:10114000F7B59C6905460E46F4B1202383F3118858
:1011500005EB8607201D0821FFF7AAFEFB685B69E7
:101160001B684C3413B1204601F0DEFC01A9204677
:1011700001F0CCFC024648B1019B3146284600F004
:101180008FF8002383F3118803B0F0BDFB685A6920
:101190001268002AF5D01B8A013B1340F1D105F1FA
:1011A0004402EAE7093138B550F82140DCB1202388
:1011B00083F31188D4F894241368527903EB8203E3
:1011C000DB689B695D6845B104216018FFF770FE1C
:1011D000294604F1140001F0CFFB2046FFF7B8FECA
:1011E000002383F3118838BD7047000000F078BFFA
:1011F000012303700023C36183620362C3624362FD
:101200000363C0E90133704738B50446202383F3F4
:10121000118800254160C0E90355C0E9055500F07B
:101220006FFF0223237085F3118838BD70B500EB82
:10123000810305465069DA600E46144618B1102243
:101240000021FFF795FDA06918B110220021FFF7DA
:101250008FFD31462846BDE8704001F01BB8000004
:10126000028902F001020281428902F001024281F8
:101270000022C0E90422826101F0A2B8F0B400EBC0
:1012800081044789E4680125A4698D403D43458177
:1012900023600023A2606360F0BC01F0BDB80000D1
:1012A000F0B400EB81040789E468012564698D408E
:1012B0003D43058123600023A2606360F0BC01F020
:1012C00037B9000070B50223002504460370C564D9
:1012D000C0E90255C0E90455856180F8345000F03A
:1012E00075FF63681B6823B129462046BDE870403E
:1012F000184770BD436802781B6880F850200522AB
:1013000002700BB10421184770470000436890F841
:1013100050201B6802700BB1052118477047000070
:1013200090F8343070B5044613B1002380F834309F
:1013300004F14402204601F065F863689B6863BBD2
:1013400094F8443013F0600515D194F8452003F06B
:101350007F0343EA022340F20232934200F0088105
:101360005BD8022B00F0DB803FD8002B00F086809A
:10137000012B00F0CE800021204601F09BFA0021D5
:10138000204601F08DFA63681B6813B106212046E0
:101390009847062384F8343070BD204698470028CB
:1013A000CED094F84B2094F84A3043EA0223E26B03
:1013B0009A4288BFE36394F94430E56B002B4FF009
:1013C000200380F2F780002D00F0E680092284F8E7
:1013D000342083F311880021D4E90E232046FFF73F
:1013E0005FFF002383F31188D6E7B3F5817F00F018
:1013F000AB80B3F5407F48D0B3F5807FBBD194F884
:101400004630012BB7D1B4F84C3023F00203C4E9C5
:101410000E55A4F84C302564C3E740F201629342B4
:101420001DD8B3F5C06F3AD2B3F5A06FA3D1B4F80D
:101430004430B3F5A06F0ED194F8463084F84E30A6
:10144000204600F01BFF63681B6813B10121204692
:101450009847032323700023C4E90E3313E0B3F548
:10146000106F32D040F60242934252D0B3F5006F73
:1014700081D104F14F03A363012324E004F14C0262
:10148000A2630222E26323648BE794F84630012BC7
:101490007FF471AFB4F84C3043F00203B7E794F82F
:1014A0004920616894F848304E6894F8471043EA40
:1014B0000223204694F84620B04700283FF45BAF53
:1014C0004368A3630368E363A5E72378042B10D183
:1014D000202383F311882046FFF7C2FE85F311888D
:1014E000636884F84F501B68032121700BB12046BC
:1014F000984794F84630002BADD084F84F30042341
:10150000237063681B68002BA5D0022120469847F2
:10151000A1E7354BA3630223E3630023B3E794F809
:1015200048301D0603F00F0120460AD500F05CFF8D
:10153000012804D002287FF41EAF2C4BEAE72C4B85
:10154000E8E700F043FFF3E794F84630002B7FF420
:1015500012AF94F8483013F00F013FF47CAF1A0635
:10156000204602D501F0BAF975E701F0ADF972E74E
:1015700094F84630002B7FF4FEAE94F8483013F018
:101580000F013FF468AF1B06204602D501F092F927
:1015900061E701F085F95EE7142284F8342083F3D3
:1015A00011882B462A4629462046FFF767FE85F319
:1015B0001188F1E65DB1152284F8342083F3118897
:1015C0000021D4E90E232046FFF758FE09E70B223D
:1015D00084F8342083F311882B462A462946204676
:1015E000FFF75EFEE3E700BF04340008FC330008A9
:1015F0000034000838B590F834300446152B39D83B
:10160000DFE803F03E38383838383E38380B2939AF
:1016100038383838383838383E3E90F84B1090F823
:101620004A20C36B42EA0122934214D2C268128A52
:10163000B3FBF2F502FB15356DB9202383F3118856
:101640002B462A462946FFF72BFE85F311880A23ED
:1016500084F834300EE0142384F83430202383F3EC
:10166000118800231A4619462046FFF707FE00237B
:1016700083F3118838BD036C03B198470023E7E773
:10168000002101F017F90021204601F009F96368F3
:101690001B6813B10621204698470623D8E70000AF
:1016A00090F83420152A38B5044617D80123934002
:1016B00040F6416213421ED113F480150FD19B02F4
:1016C0000CD50B2380F83430202383F311882B466C
:1016D0002A462946FFF7E4FD85F3118838BDC36823
:1016E0009B695B68002BF9D1036C03B19847002319
:1016F00084F83430F2E7002101F0DCF800212046C4
:1017000001F0CEF863681B6813B1062120469847A4
:101710000623EDE7024B0022C3E900339A607047CD
:1017200008260020002303748268054B1B68996813
:101730009142FBD25A680360426010605860704763
:101740000826002008B5202383F31188037C032B8F
:1017500005D0042B0DD02BB983F3118808BD436944
:1017600000221A604FF0FF334361FFF7DBFF0023D5
:10177000F2E7D0E900231A6002685360F2E7000044
:10178000002303748268054B1B6899689142FBD85B
:101790005A68036042601060586070470826002055
:1017A000054B19690874186802681A60536018615B
:1017B00001230374FEF7A8BD0826002030B54B1C9A
:1017C00087B005460A4C10D023690A4A01A800F0E8
:1017D000D3F82846FFF7E4FF049B13B101A800F0FB
:1017E00007F92369586907B030BDFFF7D9FFF8E75B
:1017F000082600204517000838B50C4D41612B69BB
:1018000081689A689142044603D8BDE83840FFF7E2
:1018100089BF1846FFF786FF01232C610146237418
:101820002046BDE83840FEF76FBD00BF0826002007
:10183000044B1A681B6990689B68984294BF00200B
:10184000012070470826002010B5084C2368206945
:101850001A6822605460012223611A74FFF790FF16
:1018600001462069BDE81040FEF74EBD0826002065
:10187000FFF7EABF82600222028270478368A3F109
:101880007C0243F80C2C026943F83C2C426943F873
:10189000382C074A43F81C2CC26843F8102C02224B
:1018A00003F8082C002203F8072CA3F11800704756
:1018B0002103000810B5202383F31188FFF7DEFF12
:1018C00000210446FFF798FF002383F31188204688
:1018D00010BD0000024B1B6958610F20FFF760BF6D
:1018E00008260020202383F31188FFF7F3BF0000B0
:1018F00008B50146202383F311880820FFF75EFF17
:10190000002383F3118808BD49B1064B42681B6967
:1019100018605A60136043600420FFF74FBF4FF018
:10192000FF307047082600200368984206D01A68E6
:101930000260506059611846FFF7F4BE704700001E
:1019400038B504460D462068844200D138BD03688E
:1019500023605C604561FFF7E5FEF4E7054B03F1AA
:101960001402C3E905224FF0FF310022C3E9071238
:10197000704700BF08260020F8B5C0E903231B4AC2
:1019800006461046022950F8145F4FF0804338BFD6
:10199000022185425B6A17460AD11362C2E90566D5
:1019A0005818C6E90055B160BDE8F84001F082B9A9
:1019B000106A1B1A5C18AB6802D3E41A2D6804E0A5
:1019C000A34202D9204401F083F9AB68A342F4D3C7
:1019D0006B68736035601E606E60B460AB681C1B22
:1019E0004FF0FF33AC60FB61F8BD00BF082600205C
:1019F00010B41B4C234653F8141F814210D0D0E979
:101A000000210A60026851609A424FF00001C160F3
:101A100003D0936881680B4493605DF8044B704772
:101A20000A68626100209A425360C86003D15DF881
:101A3000044B01F047B993688868034493604FF002
:101A40008042206A526A121A9342E6D9991A0129F1
:101A500098BF931C18445DF8044B01F039B900BFDE
:101A60000826002000207047FEE7000070470000B5
:101A70004FF0FF3070470000022906D0032906D03E
:101A80000129064818BF0020704705487047032AFF
:101A90009ABF044800EBC20000207047D43400080D
:101AA000883400080824002070B59AB001AD0646BD
:101AB00008462946144600F095F82846FFF750F9E5
:101AC000C0B2431C5B00C6E900342370032363707B
:101AD000002302341946DAB2904204F1020401D81C
:101AE0001AB070BDEA5C04F8022C04F8011C013342
:101AF000F1E7000008B5202383F311880348FFF7BE
:101B0000F7FA002383F3118808BD00BF48260020A0
:101B100010B50446052916D8DFE801F0161503169E
:101B2000161D202383F311880E4A0121FFF77EFB47
:101B300020460D4A0221FFF779FB0C48FFF7A4FA73
:101B4000002383F3118810BD202383F311880748F5
:101B5000FFF770FAF4E7202383F311880348FFF7B7
:101B600087FAEDE7083400082C34000848260020E6
:101B700038B50C4D0C4C0D492A4604F10800FFF70E
:101B800093FF05F1CA0204F110000949FFF78CFF29
:101B900005F5CA7204F118000649BDE83840FFF7A0
:101BA00083BF00BF102B00200824002058340008F9
:101BB000623400086D34000870B5044608460D46CE
:101BC000FFF7CEF8C6B22046013403780BB91846A9
:101BD00070BD32462946FFF7ADF80028F3D1012049
:101BE000F6E700002DE9F84F05460C46FFF7B8F878
:101BF0002949C6B22846FFF7DFFF08B10136F6B221
:101C000026492846FFF7D8FF08B11036F6B2632EF2
:101C10000DD8DFF88490DFF884A0214FDFF888B07A
:101C2000DFF888802E7846B92670BDE8F88F2946FF
:101C30002046BDE8F84F01F093BB252E28D107229E
:101C400049462846FFF776F840B9D8F800302360B7
:101C5000D8F80430636007350834E3E708225146BA
:101C60002846FFF767F898B90E4BA21C19780909A6
:101C70000232C95D02F8041C13F8011B01F00F01C8
:101C80005B45C95D02F8031CF0D118340835C9E77B
:101C9000267001350134C5E7F43400086D340008BE
:101CA00005350008107AFF1F1C7AFF1FFC3400085E
:101CB000BFF34F8F024AD368DB03FCD4704700BFE9
:101CC000003C024008B5094B1B7873B9FFF7F0FFE1
:101CD000074B1A69002ABFBF064A5A6002F18832D0
:101CE0005A601A6822F480621A6008BD6E2D0020C6
:101CF000003C02402301674508B50B4B1B7893B9A4
:101D0000FFF7D6FF094B1A6942F000421A611A68C0
:101D100042F480521A601A6822F480521A601A68DB
:101D200042F480621A6008BD6E2D0020003C024023
:101D30000B2870B513D80B4A0B4C137863B90B4EB4
:101D40004FF0006144F8231056F8235001330C2B58
:101D50002944F7D10123137054F8200070BD0020EE
:101D6000FCE700BFA02D0020702D002018350008D2
:101D7000014B53F820007047183500080C207047BD
:101D80000B2810B5044601D9002010BDFFF7D0FF85
:101D9000064B53F824301844C21A0BB90120F4E75B
:101DA00012680132F0D1043BF6E700BF1835000895
:101DB0000B2810B5044621D8FFF77AFFFFF782FF02
:101DC0000F4AF323D360C300DBB243F4007343F044
:101DD00002031361136943F480331361FFF768FF53
:101DE000FFF7A6FF074B53F8241000F0DDF8FFF7CC
:101DF00083FF2046BDE81040FFF7C2BF002010BDA2
:101E0000003C024018350008F8B512F001031646F0
:101E10003DD18218B2F1016F58D22D4B1B6813F0DF
:101E2000010353D02B4CFFF74DFFF323E360FFF783
:101E30003FFF40F20127032E01D9830710D0254D23
:101E40000F46401A3144CB1B012B00EB07042B69D2
:101E500022D823F001032B61FFF74EFF0120F8BDCC
:101E6000236923F44073236123693B43236151F8C1
:101E7000045B0560BFF34F8FFFF71AFF03689D42B5
:101E800007D0236923F001032361FFF735FF00200A
:101E9000E5E7043E0430CEE723F440732B612B6961
:101EA00043F4807343F001032B613B882380BFF32D
:101EB0004F8FFFF7FDFE248837F8023BA4B2A34200
:101EC000C1D02B6923F001032B61DEE71846C6E77A
:101ED00000380240003C0240084908B50B7828B1A0
:101EE0001BB9FFF7EFFE01230B7008BD002BFCD0E0
:101EF000BDE808400870FFF7FFBE00BF6E2D002050
:101F000010B50244064B0439D2B2904200D110BD44
:101F1000441C00B253F8200041F8040FE0B2F4E78B
:101F200050280040104B30B51C6F240407D41C6FA0
:101F300044F400741C671C6F44F400441C670B4C91
:101F4000236843F4807323600244094B0439D2B2FE
:101F5000904200D130BD441C00B251F8045F43F8F8
:101F60002050E0B2F4E700BF0038024000700040AB
:101F70005028004007B5012201A90020FFF7C0FF4B
:101F8000019803B05DF804FB13B50446FFF7F2FFB8
:101F9000A04206D002A9012241F8044D0020FFF71B
:101FA000C1FF02B010BD000070470000034B1B686A
:101FB0009B0042BF024B01221A70704774380240E6
:101FC000A12D0020014B1878704700BFA12D0020E3
:101FD00070470000FEE70000084A094B09498B42A0
:101FE00004D3094A0021934205D3704752F8040FE5
:101FF00043F8040BF3E743F8041BF4E7C436000886
:1020000018300020183000201830002030B5D0E9FA
:10201000154300229D6811464FF0FF3004EB421338
:1020200001329542C3F80019C3F81019C3F8080922
:10203000C3F8001BC3F8101BC3F8080BEED24FF017
:102040000113C4F81C3830BD890141F02001016141
:1020500003699B06FCD4122000F0C2BE1F4B03EBA9
:1020600080022DE9F047D2F80CC05D6DDCF8142039
:10207000461CD2F800E005EB063605EB4018516827
:1020800071450BD3D5F83428012303FA00F022EA76
:102090000000C5F834081846BDE8F087BCF81040C9
:1020A000AEEB0103A34228BF2346D8F81849A4B2D7
:1020B000B3EB840F10D894681F46A4F1040959F8B3
:1020C00004AFC6F800A0042F01D9043FF7E71C4471
:1020D0000B4494605360D2E70020DDE7A42D00207C
:1020E00010B5054C2046FFF783F84FF0A043636519
:1020F000024BA36510BD00BFA42D00206C35000865
:102100000378012B70B5054650D12A4B446D984297
:102110001BD1294B5A6B42F080025A635A6D42F030
:1021200080025A655A6D5A6942F080025A615A69B2
:1021300022F080025A610E2143205B6900F0D8FB37
:102140001E4BE3601E4BC4F800380023C4F8003E69
:10215000C02323606E6D4FF40413A3633369002B17
:10216000FCDA012333610C2000F03AFE3369DB070F
:10217000FCD4122000F034FE3369002BFCDA002678
:10218000A6602846FFF742FF6B68C4F81068DB685A
:10219000C4F81468C4F81C684BB90A4BA3614FF02B
:1021A000FF336361A36843F00103A36070BD064B76
:1021B000F4E700BFA42D0020003802404014004086
:1021C00003002002003C30C0083C30C0F8B5446D2C
:1021D000054600212046FFF737FFA96D00234FF089
:1021E00001128F68C4F834384FF00066C4F81C2818
:1021F0004FF0FF3004EB431201339F42C2F80069F5
:10220000C2F8006BC2F80809C2F8080BF2D20B68DA
:102210006A6DEB65636210231361166916F0100690
:10222000FBD1122000F0DCFDD4F8003823F4FE636B
:10223000C4F80038A36943F4402343F01003A361BA
:102240000923C4F81038C4F814380A4BEB604FF077
:10225000C043C4F8103B084BC4F8003BC4F81069F5
:10226000C4F80039EB6D03F1100243F48013EA6502
:10227000A362F8BD4835000840800010426D90F818
:102280004E10D2F8003823F4FE6343EA0113C2F87B
:10229000003870472DE9F8430EB200EB86090D4671
:1022A000D9F80C20176807F00303022B55D0032B35
:1022B00055D03E4F3E49012B18BF0F46446D690172
:1022C00063184FF0000CC3F810CB05F110034FF06A
:1022D000010C0CFA03FC9369002B42D0B2F812E017
:1022E00005F158035B014EEA070E44F803E0D4F809
:1022F0001C3843EA0C032144C4F81C380023C1F8FD
:10230000103953694FF00108691E08FA05F8ABB39C
:10231000138A928B9B08012A88BF5343C26D9E1873
:1023200042EA034301F1400204EB8202C6652946FA
:1023300053602046FFF788FED9F80C301B8A43EA29
:10234000855348356D011F436751D4F81C3843EA63
:102350000803C4F81C38BDE8F883164FAEE7164FE3
:10236000ACE704EB461EDEF8003B23F40043CEF856
:10237000003BD4F81C3823EA0C03BCE705F13F030B
:1023800004EB83030D4A5A6004EB461629462046A7
:10239000FFF75AFED6F8003923F40043C6F8003997
:1023A000D4F81C3823EA0803D3E700BF00800410E8
:1023B000008000100080081000800C100004000253
:1023C000826D1268C265FFF721BE00005831436D6F
:1023D00049015B5813F4004004D013F4001F14BFEC
:1023E00001200220704700004831436D49015B58CD
:1023F00013F4004004D013F4001F14BF0120022086
:102400007047000000EB8101CB68196A0B6813600C
:102410004B6853607047000000EB810330B5DD6806
:10242000AA691368D36019B9402B84BF4023136095
:102430006B8A1468426D1C44013CB4FBF3F46343A3
:10244000033323F0030302EB411043EAC44343F098
:10245000C043C0F8103B2B6803F00303012B09B203
:102460000ED1D2F8083802EB411013F4807FD0F877
:10247000003B14BF43F0805343F00053C0F8003BCF
:1024800002EB4112D2F8003B43F00443C2F8003B98
:1024900030BD00002DE9F041244D6E6D06EB401378
:1024A0000446D3F8087BC3F8087B38070AD5D6F86A
:1024B0001438190706D505EB84032146DB68284646
:1024C0005B689847FA071FD5D6F81438DB071BD589
:1024D00005EB8403D968CCB98B69488A5E68B6FB82
:1024E000F0F200FB12628AB91868DA6890420DD2E5
:1024F000121AC3E90024202383F311880B482146D4
:10250000FFF78AFF84F31188BDE8F081012303FA05
:1025100004F26B8923EA02036B81CB68002BF3D0B2
:1025200021460248BDE8F041184700BFA42D002015
:1025300000EB810370B5DD68436D6C692668E66069
:102540004A0156BB1A444FF40020C2F810092A6809
:1025500002F00302012A0AB20ED1D3F8080803EBF5
:10256000421410F4807FD4F8000914BF40F080506A
:1025700040F00050C4F8000903EB4212D2F8000901
:1025800040F00440C2F80009D3F83408012202FAEE
:1025900001F10143C3F8341870BD19B9402E84BF4E
:1025A0004020206020682E8A841940F00050013CB1
:1025B0001A44B4FBF6F440EAC440C6E7F8B5044652
:1025C0001E48456D05EB4413D3F80869C3F8086944
:1025D000F10717D5D5F81038DA0713D500EB8403C7
:1025E000D9684B691F68DA68974218D2D21B002756
:1025F0001A605F60202383F311882146FFF798FF5C
:1026000087F31188330617D5D5F834280123A34062
:10261000134211D02046BDE8F840FFF71FBD01234B
:1026200003FA04F2038923EA020303818B68002B77
:10263000E8D021469847E5E7F8BD00BFA42D00206B
:1026400096482DE9F84F456D6E69AB691E4016F44A
:10265000805F6E61044605D0FEF734FEBDE8F84F9A
:1026600000F052BC002E12DAD5F8003E8B489B07D2
:102670001EBFD5F8003E23F00303C5F8003ED5F891
:10268000043823F00103C5F80438FEF73FFE370590
:1026900002D58248FEF72EFEB0040CD5D5F80838D6
:1026A00013F0060FEB6823F470530CBF43F4105380
:1026B00043F4A053EB60310704D56368DB680BB1CA
:1026C00076489847F2025AD4B3020CD5D4F8548015
:1026D000DFF8C8A100274FF00109A36D9B68F9B28C
:1026E0008B4280F08780F70619D5616D0A6AC2F3C4
:1026F0000A1702F00F0302F4F012B2F5802F00F077
:10270000A180B2F5402F0AD104EB830301F580517B
:10271000DB68186A00231A469F4240F08780300326
:10272000D5F8184813D5E10302D50020FFF7B2FE13
:10273000A20302D50120FFF7ADFE630302D50220FC
:10274000FFF7A8FE270302D50320FFF7A3FE7503BA
:1027500084D5E00702D50020FFF730FFA10702D59E
:102760000120FFF72BFF620702D50220FFF726FFAB
:1027700023077FF573AF0320FFF720FF6EE7D4F840
:102780005480DFF818A100274FF00109A36D9B6862
:102790005FFA87FB5B4597D308EB4B13D3F800290F
:1027A00002F44022B2F5802F22D1D3F80029002A6A
:1027B0001EDAD3F8002942F09042C3F80029D3F87A
:1027C0000029002AFBDB5946606DFFF73DFC22899A
:1027D00009FA0BF322EA0303238104EB8B03DB6882
:1027E0009B6813B15946504698475846FFF736FC48
:1027F0000137CBE708EB4112D2F8003B03F440234A
:10280000B3F5802F10D1D2F8003B002B0CDA62898F
:1028100009FA01F322EA0303638104EB8103DB6815
:10282000DB680BB150469847013756E79C0708BF55
:102830000A68072B98BF027003F101039CBF120ABC
:10284000013069E7023304EB830201F580515268DD
:102850009069D0F808E0D0E90020A2EB000C00223B
:10286000104697420AD104EB830463689B699A6817
:102870003A449A605A6817445F6050E712F0030FB9
:1028800008BF0868944588BF8EF8000002F1010275
:1028900084BF000A0EF1010EE3E700BFA42D002063
:1028A000436D03EB4111D1F8003B43F40013C1F831
:1028B000003B7047436D03EB4111D1F8003943F4FD
:1028C0000013C1F800397047436D03EB4111D1F893
:1028D000003B23F40013C1F8003B7047436D03EB4A
:1028E0004111D1F8003923F40013C1F800397047C1
:1028F00000F1604300F01F02400903F56143090144
:102900008000C9B200F1604083F8001300F5614017
:1029100001239340C0F880310360704730B5039CB9
:102920000172043304FB0325C0E90653049B0363CF
:102930000021059BC160C0E90000C0E90422C0E994
:102940000842C0E90A11436330BD0000416A002219
:10295000C0E90411C260C0E90A226FF00101FEF76C
:10296000EFBF0000D0E90432934201D1C2680AB936
:10297000181D70470020704703691960C268013252
:10298000C260C269134482690361934224BF436AEF
:1029900003610021FEF7C8BF38B504460D46E36861
:1029A0003BB16269131D1268A3621344E362002005
:1029B00007E0237A33B929462046FEF7A5FF002811
:1029C000EDDA38BD6FF00100FBE70000C368C269B3
:1029D000013BC3604369134482694361934224BF4E
:1029E000436A436100238362036B03B11847704756
:1029F00070B52023044683F31188866A3EB9FFF739
:102A0000CBFF054618B186F31188284670BDA36A2E
:102A1000E26A13F8015BA362934202D32046FFF7F8
:102A2000D5FF002383F31188EFE700002DE9F84F6D
:102A300004460E4690469946202787F311880025C4
:102A4000AA46D4F828B0BBF1000F09D14946204668
:102A5000FFF7A2FF20B18BF311882846BDE8F88F5D
:102A6000D4E90A13A8EB050B5B1A9B4528BF9B46CC
:102A7000BBF1400F1BD9334601F1400251F8040B62
:102A800043F8040B9142F9D1A36A40334036A36264
:102A90004035D4E90A239A4202D32046FFF796FF35
:102AA0008AF311884545D8D287F31188C9E73046A3
:102AB0005A46FEF735F9A36A5B445E44A3625D445F
:102AC000E7E7000010B5029C0172043304FB032108
:102AD000C0E906130023C0E90A33039B0363049B88
:102AE000C460C0E90000C0E90422C0E908424363B1
:102AF00010BD0000026AC260426AC0E904220022DE
:102B0000C0E90A226FF00101FEF71ABFD0E90423E1
:102B10009A4201D1C26822B9184650F8043B0B60B2
:102B20007047002070470000C368C2690133C3606A
:102B30004369134482694361934224BF436A4361FA
:102B40000021FEF7F1BE000038B504460D46E368EB
:102B50003BB123691A1DA262E2691344E3620020BB
:102B600007E0237A33B929462046FEF7CDFE002838
:102B7000EDDA38BD6FF00100FBE700000369196072
:102B8000C268013AC260C269134482690361934218
:102B900024BF436A036100238362036B03B11847B8
:102BA0007047000070B5202304460E4683F3118859
:102BB000856A35B91146FFF7C7FF10B185F3118853
:102BC00070BDA36A1E70A36AE26A01339342A362D6
:102BD00004D3E16920460439FFF7D0FF002080F3D9
:102BE0001188EDE72DE9F84F04460D4691469A46C7
:102BF0004FF0200888F311880026B346A76A4FB922
:102C000051462046FFF7A0FF20B187F311883046D8
:102C1000BDE8F88FD4E90A07A9EB06033F1A9F42E3
:102C200028BF1F46402F1BD905F1400355F8042B40
:102C300040F8042B9D42F9D1A36A4033A362403689
:102C4000D4E90A239A4204D3E16920460439FFF704
:102C500095FF8BF311884E45D9D288F31188CDE7C3
:102C600029463A46FEF75CF8A36A3B443D44A3621A
:102C70003E44E5E7D0E904239A4217D1C3689BB1EB
:102C8000836A8BB1043B9B1A0ED01360C368013B6F
:102C9000C360C3691A44836902619A4224BF436ACC
:102CA0000361002383620123184670470023FBE77A
:102CB00000F06CB94FF08043002258631A61022281
:102CC000DA6070474FF080430022DA6070470000FE
:102CD0004FF0804358637047FEE7000010B5174C73
:102CE000FEF718FDFEF73AFE802215492046FEF752
:102CF000C1FD012344F8180C0374124B124AD96821
:102D000021F4E0610904090C0A431049DA60CA6839
:102D100042F08072CA600E490A6842F001020A60FD
:102D20001022DA77202283F82220002383F31188EF
:102D300062B60848BDE81040FEF7BCBD3026002052
:102D40007835000800ED00E00003FA05F0ED00E042
:102D5000001000E0803500082DE9F84F1F4C4FF0BF
:102D60000008656904F11407C1464FF08043266AE4
:102D70005B6AAA689E1B96421DD34FF0200AAA6880
:102D8000236AD5F80CB0134423622B68BB425F6002
:102D9000A6EB02066361C5F80C8001D1FFF792FF34
:102DA00089F311882869D8478AF311886569AB6867
:102DB0009E42E4D2D9E76269BA420CD0916823629C
:102DC0008E1B9660A86802282CBF1818981CBDE8B6
:102DD000F84FFFF77DBFBDE8F88F00BF0826002041
:102DE000034B59685A68521A9042FBD8704700BF8B
:102DF000001000E04B6843608B688360CB68C36061
:102E00000B6943614B6903628B6943620B68036022
:102E10007047000008B5224B22481A6940F2FF11A2
:102E20000A431A611A6922F4FF7222F001021A6140
:102E30001A691A6B0A431A631A6D0A431A651A4A09
:102E40001B6D1146FFF7D6FF184802F11C01FFF772
:102E5000D1FF174802F13801FFF7CCFF154802F106
:102E60005401FFF7C7FF144802F17001FFF7C2FFDA
:102E7000124802F18C01FFF7BDFF114802F1A801D1
:102E8000FFF7B8FF0F4802F1C401FFF7B3FF0E4888
:102E900002F1E001FFF7AEFFBDE8084000F0E0B846
:102EA0000038024000000240A03500080004024043
:102EB00000080240000C02400010024000140240D2
:102EC00000180240001C02400020024008B500F03B
:102ED00037FAFFF703FFFFF769F8BDE80840FEF790
:102EE00047BE000070470000064A536823F0010304
:102EF0005360EFF30983683383F30988002383F376
:102F00001188704730EF00E010B5202383F311885B
:102F1000104B5B6813F4006318D0F1EE103AEFF336
:102F200009844FF0807344F84C3C0B4BDB6844F849
:102F3000083CA4F1680383F30988FEF779FC18B113
:102F4000064B44F8503C10BD054BFAE783F311885B
:102F5000F9E700BF00ED00E030EF00E031030008CA
:102F6000340300084FF0804310B51A69920708D562
:102F700000241C61202383F31188FFF7EDFE84F306
:102F80001188BDE81040FFF7BFBF0000104B1A6C5E
:102F900042F001021A641A6E42F001021A660D4AEA
:102FA0001B6E936843F0010393604FF080435322FC
:102FB0009A624FF0FF32DA6200229A615A63DA6055
:102FC0005A6001225A6108211A601C20FFF790BC48
:102FD00000380240002004E01F4B1A696FEAC25219
:102FE0006FEAD2521A611A69C2F308021A614FF0ED
:102FF000FF301A695A69586100215A6959615A6942
:103000001A6A62F080521A621A6A02F080521A62D8
:103010001A6A5A6A58625A6A59625A6A1A6C42F0B3
:1030200080521A641A6E42F080521A661A6E0B4A67
:10303000106840F480701060186F00F44070B0F5B4
:10304000007F1EBF4FF4803018671967536823F460
:103050000073536000F054B9003802400070004023
:10306000304B4FF080521A642F4A4FF440411160A8
:103070001A6842F001021A601A689207FCD59A6831
:1030800022F003029A60274B19469A6812F00C024C
:10309000FBD1186800F0F90018609A601A6842F4D1
:1030A00080321A600B689B03FCD54B6F43F0010321
:1030B0004B671C4B5A6F9007FCD51C4A5A601A6824
:1030C00042F080721A60184A53685904FCD5154BB7
:1030D0001A689201FCD5164A9A60164B1A68164B6C
:1030E0009A42164B1BD1164A1168164A914216D1C4
:1030F00040F205121A600B4B9A6842F002029A6085
:103100009A6802F00C02082AFAD15A6C42F4804202
:103110005A645A6E42F480425A665B6E704740F2BF
:103120000572E7E70038024000700040085440078D
:1031300000948838002004E011640020003C024024
:1031400000ED00E041C20F41084A08B5516913681B
:103150000B4003F00103536123B1054A13680BB11F
:1031600050689847BDE80840FFF7CEBE003C0140DC
:1031700088250020084A08B5516913680B4003F000
:103180000203536123B1054A93680BB1D068984795
:10319000BDE80840FFF7B8BE003C0140882500208C
:1031A000084A08B5516913680B4003F004035361E2
:1031B00023B1054A13690BB150699847BDE808402F
:1031C000FFF7A2BE003C014088250020084A08B550
:1031D000516913680B4003F00803536123B1054A9A
:1031E00093690BB1D0699847BDE80840FFF78CBEE2
:1031F000003C014088250020084A08B55169136841
:103200000B4003F01003536123B1054A136A0BB15D
:10321000506A9847BDE80840FFF776BE003C014081
:1032200088250020174B10B55A691C68144004F417
:1032300078725A61A30604D5134A936A0BB1D06A17
:103240009847600604D5104A136B0BB1506B984732
:10325000210604D50C4A936B0BB1D06B9847E2055D
:1032600004D5094A136C0BB1506C9847A30504D5DB
:10327000054A936C0BB1D06C9847BDE81040FFF73E
:1032800043BE00BF003C0140882500201A4B10B50A
:103290005A691C68144004F47C425A61620504D5E2
:1032A000164A136D0BB1506D9847230504D5134A88
:1032B000936D0BB1D06D9847E00404D50F4A136E9F
:1032C0000BB1506E9847A10404D50C4A936E0BB114
:1032D000D06E9847620404D5084A136F0BB1506F43
:1032E0009847230404D5054A936F0BB1D06F9847D4
:1032F000BDE81040FFF708BE003C014088250020D3
:10330000062108B50846FFF7F3FA06210720FFF764
:10331000EFFA06210820FFF7EBFA06210920FFF754
:10332000E7FA06210A20FFF7E3FA06211720FFF744
:10333000DFFA06212820BDE80840FFF7D9BA0000CF
:1033400008B5FFF749FEFDF7A7FDFDF74FFFFDF7B5
:1033500029FEFFF7C7FDBDE80840FFF7A9BC000044
:10336000034611F8012B03F8012B002AF9D170470D
:10337000121012131211000053544D3332463F3FC6
:103380003F00000000000000783300083F0000000C
:1033900013040000B43300083F00000019040000CB
:1033A000BE3300083F00000021040000C8330008BD
:1033B0003F00000053544D333246343078005354AC
:1033C0004D3332463432780053544D333246343420
:1033D00036585800000000001D0F0008090F0008B3
:1033E000450F0008310F00083D0F0008290F0008A5
:1033F000150F0008010F0008A10F000800000000D1
:1034000001000000000000000200000000000000B9
:103410003D110008A511000840004000E02A0020EE
:10342000F02A00200200000000000000030000005D
:1034300000000000E911000800000000100000007A
:10344000002B002000000000010000000000000030
:10345000A42D0020010102004172647550696C6F57
:10346000740025424F415244252D424C00255345BE
:103470005249414C25000000111B0008791A000830
:10348000B5100008F51A0008430000009034000849
:1034900009024300020100C03209040000010202D7
:1034A000010005240010010524010001042402028A
:1034B0000524060001070582030800FF0904010036
:1034C000020A000000070501024000000705810212
:1034D0004000000012000000DC340008120110015E
:1034E00002000040091241570002010203010000DE
:1034F0000403090425424F41524425005375636378
:103500006578463400303132333435363738394116
:1035100042434445460000000040000000400000D7
:103520000040000000400000000001000000020018
:103530000000020000000200000002000000020083
:10354000000002000000020000000000211300083B
:10355000F5150008A116000840004000042E0020C8
:10356000042E002001000000142E00208000000026
:1035700040010000030000006D61696E0000000062
:1035800098350008202E002018300020010000008F
:10359000D92C00080000000069646C650000000080
:1035A0000000800200000000AAAAAAAA00000000F1
:1035B000FFFF00000000000000A00A00000400005F
:1035C00000000000AAAAAAAA00000000DFFF000075
:1035D00000000000000000000000000000000000EB
:1035E000AAAAAAAA00000000FFFF00000000000035
:1035F000000000000000000000000000AAAAAAAA23
:1036000000000000FFFF00000000000000000000BC
:103610000000000000000000AAAAAAAA0000000002
:10362000FFFF00000000000000000000000000009C
:1036300000000000AAAAAAAA00000000FFFF0000E4
:10364000000000000000000000000000000000007A
:10365000AAAAAAAA00000000FFFF000000000000C4
:103660000000000000000000000000000A00000050
:103670000000000003000000000000000000000047
:10368000000000000000000000000000000000003A
:10369000000000000000000000000000000000002A
:1036A000FF0096000000000804000000F03400084D
:1036B000000000000000000000000000000000000A
:0836C000000000000000000002
:00000001FF
